:100000000C942A000C9447000C9447000C94470071
:100010000C9447000C9447000C9447000C94470044
:100020000C9447000C9447000C9447000C94470034
:100030000C9447000C9447000C9447000C94470024
:100040000C9447000C9447000C9447000C94470014
:100050000C94470011241FBECFE5D4E0DEBFCDBF16
:1000600010E0A0E6B0E0EAE2FEE002C005900D92EA
:10007000A23BB107D9F711E0A2EBB0E001C01D929D
:10008000A330B107E1F70E947E060C9414070C948C
:100090000000CF93DF93CDB7DEB7EBE3F0E0108243
:1000A000EAE3F0E01082E8E3F0E01082E7E3F0E05A
:1000B0008FE08083E5E3F0E01082E4E3F0E010827B
:1000C000E2E3F0E01082E1E3F0E082E08083DF91A0
:1000D000CF910895CF93DF93CDB7DEB726970FB6B4
:1000E000F894DEBF0FBECDBF6B837C838D839E8370
:1000F0008B819C81AD81BE81880F991FAA1FBB1F78
:10010000880F991FAA1FBB1F880F991FAA1FBB1F0B
:10011000880F991FAA1FBB1F9C01AD0180E094E2CC
:10012000A4EFB0E0BC01CD010E94F206DA01C901E2
:1001300001979A838983E0E4F0E089819927892FE8
:10014000990F990B8083E9E2F0E089818083AAE22C
:10015000B0E0EAE2F0E0808188618C93A0E4B0E056
:10016000E0E4F0E0808186688C9326960FB6F894E0
:10017000DEBF0FBECDBFDF91CF910895CF93DF9348
:10018000CDB7DEB722970FB6F894DEBF0FBECDBF56
:10019000EBE2F0E08081882344F4ECE2F0E080813F
:1001A000282F33273A83298302C01A821982898132
:1001B0009A8122960FB6F894DEBF0FBECDBFDF91B5
:1001C000CF910895CF93DF93CDB7DEB721970FB6C8
:1001D000F894DEBF0FBECDBF8983EBE2F0E08081F3
:1001E0009927807290700097C1F3ECE2F0E089816A
:1001F000808321960FB6F894DEBF0FBECDBFDF918E
:10020000CF910895CF93DF93CDB7DEB723970FB685
:10021000F894DEBF0FBECDBF9B838A83198203C0D3
:1002200089818F5F8983898199279C018A819B813C
:10023000F901E80FF91F8081882391F789819927B7
:1002400023960FB6F894DEBF0FBECDBFDF91CF91DE
:100250000895CF93DF93CDB7DEB725970FB6F89407
:10026000DEBF0FBECDBF9D838C838C819D810E949C
:1002700002018B831A8210C08A8199279C018C818C
:100280009D81F901E80FF91F8081898389810E948E
:10029000E2008A818F5F8A839A818B81981760F34D
:1002A000EC81FD81108225960FB6F894DEBF0FBE5B
:1002B000CDBFDF91CF910895CF93DF93CDB7DEB758
:1002C00025970FB6F894DEBF0FBECDBF9D838C83FC
:1002D0008C819D810E9402018B831A8210C08A81C9
:1002E00099279C018C819D81F901E80FF91F80817C
:1002F000898389810E94E2008A818F5F8A839A8143
:100300008B81981760F3EC81FD8110828DE00E9453
:10031000E2008AE00E94E20025960FB6F894DEBF64
:100320000FBECDBFDF91CF910895CF93DF93CDB7AF
:10033000DEB78DE00E94E2008AE00E94E200DF91D9
:10034000CF910895CF93DF93CDB7DEB764970FB603
:10035000F894DEBF0FBECDBF0E94950183EB90E005
:100360009A838983E0E6F0E0FC83EB83F9E1FD8387
:10037000EB81FC8100808B819C8101969C838B8327
:10038000E981FA81008289819A8101969A83898321
:100390009D8191509D83ED81EE2351F783EB90E099
:1003A0000E945C0183EB90E09F838E83E9E7F0E09D
:1003B000F987E887F9E1FA87E885F985008088857B
:1003C0009985019699878887EE81FF8100828E81C9
:1003D0009F8101969F838E839A8591509A87EA85A3
:1003E000EE2351F783EB90E00E945C0183EB90E0F9
:1003F0009C878B87E2E9F0E0FE87ED87F9E1FF87D4
:10040000ED85FE8500808D859E8501969E878D8772
:10041000EB85FC8500828B859C8501969C878B876C
:100420009F8591509F87EF85EE2351F783EB90E0F6
:100430000E945C0183EB90E0998B888BE0E6F0E012
:10044000FB8BEA8BF9E1FC8BEA89FB8900808A89C6
:100450009B8901969B8B8A8BE889F9890082888920
:1004600099890196998B888B9C8991509C8BEC89FA
:10047000EE2351F783EB90E00E945C0164960FB687
:10048000F894DEBF0FBECDBFDF91CF910895CF931B
:10049000DF93CDB7DEB726970FB6F894DEBF0FBE59
:1004A000CDBF19820E94950183EB90E09B838A83E4
:1004B000EBEAF0E0FD83EC83F7E0FE83EC81FD8165
:1004C00000808C819D8101969D838C83EA81FB81D4
:1004D00000828A819B8101969B838A839E819150B1
:1004E0009E83EE81EE2351F783EB90E00E945C0146
:1004F0000E94950126960FB6F894DEBF0FBECDBFC1
:10050000DF91CF910895CF93DF93CDB7DEB72997D1
:100510000FB6F894DEBF0FBECDBF198203C00E9494
:10052000BE00898389818823D1F38981873529F4A5
:1005300081E090E0998788875EC08981873729F4B8
:1005400082E090E09987888756C08981823529F4B6
:1005500083E090E0998788874EC08981823729F4AB
:1005600084E090E09987888746C01F828981833420
:1005700011F491E09F831E828981833611F481E01A
:100580008E838F819E81892B882329F085E090E0DE
:100590009987888730C01D8289818F3411F491E05A
:1005A0009D831C8289818F3611F481E08C838D813B
:1005B0009C81892B882329F086E090E099878887A1
:1005C0001AC01B828981833511F491E09B831A82C2
:1005D0008981833711F481E08A838B819A81892B09
:1005E000882329F087E090E09987888704C088E015
:1005F00090E0998788878885998529960FB6F89421
:10060000DEBF0FBECDBFDF91CF910895CF93DF93B3
:10061000CDB7DEB7E4970FB6F894DEBF0FBECDBFFF
:100620008A871C8281E089831A820DC08A81282FE3
:100630003327CE010596FC01E20FF31F80E3808390
:100640008A818F5F8A838A81853080F31A828A85C6
:10065000282F33273AAB29AB89A99AA98130910574
:1006600009F454C029A93AA92230310509F43CC142
:10067000E8C10E94BE008C833C813BAB8BA98823E0
:1006800011F091E09BAB2BA928AB1FA68C818A307F
:1006900011F031E03FA788A99FA58923282F332790
:1006A0003EA72DA71CA61BA68C818D3021F081E0D2
:1006B00090E09CA78BA72DA53EA58BA59CA52823E4
:1006C000392389819927822393230097F9F01AA669
:1006D0008C81803311F091E09AA719A68C81813327
:1006E00011F021E029A78AA539A58323882309F0E1
:1006F00019828A81282F3327CE010596FC01E20F4B
:10070000F31F8C8180838A818F5F8A8318A68C81F6
:100710008A3011F081E088A71FA28C818D3011F002
:1007200091E09FA388A52FA18223282F33273EA3E2
:100730002DA31CA21BA28A81853020F481E090E0C9
:100740009CA38BA32DA13EA18BA19CA1282339237F
:100750008981992782239323009709F08ACF1AA2CF
:100760008A81853011F491E09AA319A289818823A6
:1007700011F421E029A38AA139A1832B882319F040
:100780000E9447025EC18D81813341F4A8E3B0E04D
:10079000E8E3F0E0808181608C9308C0A8E3B0E0DA
:1007A000E8E3F0E090818EEF89238C938E81813392
:1007B00041F4A8E3B0E0E8E3F0E0808182608C934C
:1007C00008C0A8E3B0E0E8E3F0E090818DEF892372
:1007D0008C938F81813341F4A8E3B0E0E8E3F0E04B
:1007E000808184608C9308C0A8E3B0E0E8E3F0E087
:1007F00090818BEF89238C938885813341F4A8E322
:10080000B0E0E8E3F0E0808188608C931AC1A8E34F
:10081000B0E0E8E3F0E0908187EF89238C9311C189
:100820000E94BE008C838C818CAB9CA9992311F013
:1008300021E02CAB3CA938A31F8E8C818A3011F0AB
:1008400081E08F8F88A19F8D8923282F33273E8FAA
:100850002D8F1C8E1B8E8C818D3021F081E090E0DD
:100860009C8F8B8F2D8D3E8D8B8D9C8D28233923D6
:1008700089819927822393230097B1F18A818F5F21
:100880008A838C818B831A8E198E8B81803320F41E
:1008900021E030E03A8F298F188E8B818A3310F057
:1008A00031E0388F1F8A8B81813410F481E08F8B87
:1008B000888D9F8989239927298D3A8D282B392B5B
:1008C0003E8B2D8B1C8A1B8A8B81873420F081E024
:1008D00090E09C8B8B8B8D899E892B893C89822B08
:1008E000932B009709F019821A8A8C818A3011F0B3
:1008F00031E03A8B198A8C818D3011F081E0898B3F
:100900008A8999898923282F3327388B2F871E8638
:100910001D868A81823020F481E090E09E878D8759
:100920002F8538898D859E852823392389819927AC
:1009300082239323009709F073CF8B818C831C86CD
:100940008981882311F491E09C871B868A818230FB
:1009500011F421E02B878C853B85832B882319F0AC
:100960000E9447026EC01A828C818A3320F48C81E7
:1009700080538C8317C08C8187538C8313C08A81EA
:10098000282F33278C818170482F405DCE0105963A
:10099000FC01E20FF31F40838A818F5F8A838C8181
:1009A00086958C838C81882351F78885813341F427
:1009B000A8E3B0E0E8E3F0E0808181608C9308C0B8
:1009C000A8E3B0E0E8E3F0E090818EEF89238C9318
:1009D0008F81813341F4A8E3B0E0E8E3F0E0808167
:1009E00082608C9308C0A8E3B0E0E8E3F0E0908177
:1009F0008DEF89238C938E81813341F4A8E3B0E09D
:100A0000E8E3F0E0808184608C9308C0A8E3B0E064
:100A1000E8E3F0E090818BEF89238C938D81813323
:100A200041F4A8E3B0E0E8E3F0E0808188608C93D3
:100A300008C0A8E3B0E0E8E3F0E0908187EF892305
:100A40008C93E4960FB6F894DEBF0FBECDBFDF9156
:100A5000CF910895CF93DF93CDB7DEB724970FB62C
:100A6000F894DEBF0FBECDBF8A8319828A81282FFA
:100A700033273C832B838B819C818130910539F016
:100A80002B813C812230310509F43EC076C0E9E378
:100A9000F0E08081992784709070009721F481E3C1
:100AA0000E94E20003C080E30E94E200E9E3F0E07C
:100AB0008081992782709070009721F481E30E94D1
:100AC000E20003C080E30E94E200E9E3F0E08081FD
:100AD000992781709070009721F481E30E94E200D1
:100AE00003C080E30E94E200E0E3F0E08081992708
:100AF00084709070009721F481E30E94E2003DC071
:100B000080E30E94E20039C0E9E3F0E080819927A8
:100B100084709070009719F48981885F8983E9E374
:100B2000F0E08081992782709070009719F4898194
:100B30008C5F8983E9E3F0E0808199278170907070
:100B4000009719F489818E5F8983E0E3F0E080816A
:100B5000992784709070009719F489818F5F898339
:100B600089818A3020F48981805D898303C08981ED
:100B7000895C898389810E94E20024960FB6F894EB
:100B8000DEBF0FBECDBFDF91CF910895CF93DF932E
:100B9000CDB7DEB726970FB6F894DEBF0FBECDBF38
:100BA0008A838A81282F33273E832D838D819E81DE
:100BB00082309105A9F02D813E812330310509F461
:100BC0007AC08D819E818130910509F08EC0A8E3A5
:100BD000B0E0E8E3F0E0908180EF89238C9385C05A
:100BE000A8E3B0E0E8E3F0E080818F608C937DC003
:100BF0000E94BE008983E9E3F0E080819927847038
:100C00009070009749F0A8E3B0E0E8E3F0E090814D
:100C10008EEF89238C9307C0A8E3B0E0E8E3F0E00F
:100C2000808181608C93E9E3F0E080819927827074
:100C30009070009749F0A8E3B0E0E8E3F0E090811D
:100C40008DEF89238C9307C0A8E3B0E0E8E3F0E0E0
:100C5000808182608C93E9E3F0E080819927817044
:100C60009070882349F0A8E3B0E0E8E3F0E09081D9
:100C70008BEF89238C9307C0A8E3B0E0E8E3F0E0B2
:100C8000808184608C93E0E3F0E080819927847018
:100C90009070009749F0A8E3B0E0E8E3F0E09081BD
:100CA00087EF89238C9307C0A8E3B0E0E8E3F0E086
:100CB000808188608C931C828981833711F091E058
:100CC0009C831B828981833511F021E02B838C81E9
:100CD0003B818323882309F08BCFA8E3B0E0E8E3CE
:100CE000F0E0908180EF89238C9326960FB6F894DC
:100CF000DEBF0FBECDBFDF91CF910895CF93DF93BD
:100D0000CDB7DEB722970FB6F894DEBF0FBECDBFCA
:100D10000E94490060E875E280E090E00E946A006D
:100D200000C01092B2000E94A20104C00E9483027F
:100D30008093B2008091B2008823C1F38091B20009
:100D4000282F33273A83298389819A81843091051A
:100D5000B1F129813A812530310584F489819A8164
:100D60008230910521F129813A81233031051CF52A
:100D700089819A8181309105B1F0D3CF29813A815F
:100D80002630310521F189819A8186309105DCF088
:100D900029813A8127303105F1F089819A818830A3
:100DA0009105E9F0BECF81E00E940603BACF82E050
:100DB0000E940603B6CF81E00E942A05B2CF82E0EE
:100DC0000E942A05AECF81E00E94C605AACF82E02C
:100DD0000E94C605A6CF83E00E94C605A2CF0E944E
:100DE00047029FCFA1E21A2EAA1BBB1BFD010DC01B
:100DF000AA1FBB1FEE1FFF1FA217B307E407F507CB
:100E000020F0A21BB30BE40BF50B661F771F881FA6
:100E1000991F1A9469F760957095809590959B013C
:0A0E2000AC01BD01CF010895FFCF22
:100E2A002A2A2A2A2A2A2A2A2A2A2A2A2A2A2A2A18
:100E3A002A2A2A2A2A2A2A2A002A20202020415617
:100E4A005220494F20434F4E54524F4C20202020CD
:100E5A002A002A2028432920323030372C204F4CB0
:100E6A00494D4558204C7464202A004552524F522D
:020E7A00210055
:00000001FF
